:10000000BE28FF3FFF3FFF3FA60003088301B60065
:100010000A08C7008A018D2B820041346A34753486
:1000200073347434653420346C346134203468346F
:100030006F34723461343A3400340000313428347F
:10004000313430343134303431343134303431348B
:1000500030343134463465346334683461342034A8
:100060007934203468346F3472346134003441346C
:100070006A34753473347434653420346C346134C8
:100080002034663465346334683461343A3400347F
:1000900041346A34753473347434653420346534CF
:1000A0006C3420346434693461343A340034463476
:1000B0004534433448344134203449344E34433495
:1000C0004F34523452344534433454344134003480
:1000D0004134423453344F344C3455345434413425
:1000E000003420342034203420344C3455344E3401
:1000F0004534533400342034203420344D344134DA
:10010000523454344534533400344D344934453436
:10011000523443344F344C34453453340034203457
:10012000203420344A34553445345634453453341D
:1001300000342034203456344934453452344E345B
:100140004534533400342034203420345334413483
:100150004234413444344F34003420342034443465
:100160004F344D3449344E3447344F3400347134B5
:100170007B3485348F349934A334AD340F30D500BB
:100180000D122130C2008F30D800860187018B30DC
:100190007627D20000307627A10001307627A20012
:1001A00002307627A30003307627A4000430762798
:1001B000AA0005307627AB0006307627AC00073062
:1001C0007627AD0008307627AE0009307627AF00DD
:1001D0000A307627B5001430C8000A161D230A30ED
:1001E000CA000A30CB00FF30CD00FF30CE00A91688
:1001F0008A307627003C0319A91280308B008316C1
:1002000002308100850187150716871487150714AA
:1002100086018713071387120712071180309F008A
:10022000FF3092000514831217129712EF309500D9
:100230009214121597151715332733270A30A70084
:100240007D30A8003C30A5000A167A200E307627B3
:10025000003C031D2E29FC258227CD2781010B118F
:100260008B163A27FC25CF254E242918CF2529198E
:100270009F27A919CD27291A5121A91F4A29871C6F
:100280004621871D4621071C46213529A9134E24E6
:10029000CC100800871CDD2F071C5529871D521420
:1002A0003529FC25CF25291208003A274D303D2756
:1002B00004304B27683015270F304B276D303D2712
:1002C00040304B27123076273D270B3076271E27EC
:1002D0000C3076271E272C303D270D3076271E2721
:1002E0004B304B27133076273D270F3076271E27BC
:1002F000103076271E272C303D27113076271E27F9
:100300004E24EF30C400FF30B100FF303230071C04
:100310009429871D4D2B871C3129B20B8729B10BDE
:100320008529C40B832931293A274D303D270530D3
:100330004B27753015270F304B276D303D27403048
:100340004B27163076273D27173076271E27183083
:1003500076271E272C303D27193076271E274B3055
:100360004B271A3076273D271B3076271E271C3057
:1003700076271E272C303D271D3076271E274E243A
:10038000EF30C400FF30B100FF303230071CD329FA
:10039000871C3129871DCF2FB20BC629B10BC42969
:1003A000C40BC22931293A274D303D2705304B2750
:1003B0007E3015270F304B276D303D2740304B27BF
:1003C0001E3076273D271F3076271E2720307627C0
:1003D0001E272C303D27213076271E274B304B27F8
:1003E000223076273D27233076271E272430762794
:1003F0001E272C303D27253076271E274E24EF3030
:10040000C400FF30B100FF303230071C122A871CB5
:100410003129871DD12FB20B052AB10B032AC40B3A
:10042000012A31293A274D303D2703304B278530AB
:1004300015270F304B276D303D2740304B27263096
:1004400076273D27273076271E27283076271E2738
:100450002C303D27293076271E274B304B272A305A
:1004600076273D272B3076271E272C3076271E2710
:100470002C303D272D3076271E274E24EF30C40028
:10048000FF30B100FF303230071C512A871C312960
:10049000871DD32FB20B442AB10B422AC40B402A2A
:1004A00031293A274D303D2705304B27923015270B
:1004B0000F304B276D303D2740304B272E307627AD
:1004C0003D272F3076271E27303076271E272C30E9
:1004D0003D27313076271E274B304B273230762789
:1004E0003D27333076271E27343076271E272C30C1
:1004F0003D27353076271E274E24EF30C400FF30CD
:10050000B100FF303230071C902A871C3129871D2B
:10051000D52FB20B832AB10B812AC40B7F2A312934
:100520003A274D303D2704304B279B3015270F309D
:100530004B276D303D2740304B27363076273D27FF
:10054000373076271E27383076271E272C303D2758
:10055000393076271E274B304B273A3076273D27F8
:100560003B3076271E273C3076271E272C303D2730
:100570003D3076271E274E24EF30C400FF30B100F7
:10058000FF303230071CCF2A871C3129871DD72F17
:10059000B20BC22AB10BC02AC40BBE2A31293A279A
:1005A0004D303D2705304B27A63015270F304B2700
:1005B0006D303D2740304B273E3076273D273F307A
:1005C00076271E27403076271E272C303D274130C6
:1005D00076271E274B304B27423076273D27433066
:1005E00076271E27443076271E272C303D2745309E
:1005F00076271E274E24EF30C400FF30B100FF30B5
:100600003230071C0E2B871C3129871DD92FB20BC6
:10061000012BB10BFF2AC40BFD2A31293A274D309B
:100620003D2704304B27AF3015270F304B276D3057
:100630003D2740304B27463076273D2747307627E9
:100640001E27483076271E272C303D274930762735
:100650001E274B304B274A3076273D274B307627D5
:100660001E274C3076271E272C303D274D3076270D
:100670001E274E24EF30C400FF30B100FF3032306F
:10068000071C3129871C3129871DDB2FB20B402B1A
:10069000B10B3E2BC40B3C2B31295F26502355292F
:1006A0000730B200FF30B000FF30B10087190800FA
:1006B000B10B562BB00B542BB20B522B82270800D8
:1006C00052143A2702304B272A3015274E24871C14
:1006D000672BEF30C400FF30B100FF303230871C91
:1006E0007A2B871D7C2BB20B6F2BB10B6D2BC40BA0
:1006F0006B2B31290A16AC2C5F260730B000FF3077
:10070000B100FF30B2008719672BB20B832BB10BFE
:10071000812BB00B7F2B572431290A16722CC20B68
:100720009B2B1A3081072130C200D80B9B2B003045
:1007300081078F30D80006308107D00BA72BFF3000
:10074000D000CF0BA72B043081070330CF00A80BBC
:10075000412C7D30A800A70B412C0A30A700C80B04
:10076000B42B29161430C800A50B402C3C30A50032
:100770002914A40A24080A3C031D3C2CA401A30A42
:100780002308063C031D3C2CA301A20A22080A3CB4
:10079000031DCC2BA201A10A210E2204243C031923
:1007A000D22B3C2CA915A201B50A3508073C031928
:1007B000B501A101AB0A2B080A3C031DE12BAB01DB
:1007C000AA0A2C0E2D04023C031D0D2C2E08B70086
:1007D0000319FA2BA9140230A906B70BEC2BA918A0
:1007E000FA2B02302F020319062C06302F020319B0
:1007F000062C0D2CAF080319062C04302F02031908
:10080000062C08302F020319062C0D2C2A0E2B045F
:100810000310293C03183C2C1D2C2C08013C031D03
:10082000132C2730142C1D302D070C20B3002A0E5A
:100830002B040310330203183C2CAA010130AB0037
:10084000AD0A2D080A3C031D272CAD01AC0A2C0E65
:100850002D04133C031D3C2CAC010130AD00AF0A4C
:100860002F080A3C031D3C2CAF01AE0A2E080A3C9F
:10087000031D3C2CAE013C2CA91E402C0A16262C34
:100880002915A91B4C24A91F071247088A003608FE
:10089000830026080B1109000A163A2C5F26871CD4
:1008A0004F2C871D512C071C532C5F2608008316E4
:1008B000811683123A270D30152745304B27210822
:1008C0001E2722081E273A303D2723081E2724080A
:1008D0001E2745304B270E3044274E24071C752C0D
:1008E000871C982C871D802C6E2CA10A2108033CA4
:1008F0000319A10121081E2745304B274E246E2CD9
:100900004E240C3044273A27210E22040310233CA6
:1009100003188C2CA101A2010A30A7007D30A80089
:100920003C30A50081010B1183168112831208004F
:1009300046304B274E24071CA22C871CAD2C871D4C
:10094000802C9B2CA20A22080A3C0319A20122082F
:100950001E2746304B274E249B2C48304B274E24D5
:10096000071CB72C871CC22C871D802CB02CA30A17
:100970002308063C0319A30123081E2748304B27F0
:100980004E24B02C49304B274E24071CCC2C871CFE
:10099000D72C871D802CC52CA40A24080A3C0319D7
:1009A000A40124081E2749304B274E24C52C3A2782
:1009B0003730152744304B27BE2544304B274E2473
:1009C000871CF12C071CE52CE02CA915AA0A2A0883
:1009D000043C0319AA012A081E2744304B274E2441
:1009E000E02C45304B274E24871C052D071CF92C85
:1009F000F42CA915AB0A2B080A3C0319AB012B08F0
:100A00001E2745304B274E24F42C47304B274E24CD
:100A1000871C192D071C0D2D082DA915AC0A2C08B3
:100A2000023C0319AC012C081E2747304B274E24EB
:100A3000082D48304B274E24871C332D071C212DB1
:100A40001C2DA915AD0A2D080A3C0319AD012D086E
:100A50001E2748304B274E241C2D3A275730152788
:100A600020304E27D72C4A304B274E24871C472D49
:100A7000071C3B2D362DA915AE0A2E080A3C03197A
:100A8000AE012E081E274A304B274E24362D4B3000
:100A90004B274E24871C5B2D071C4F2D4A2DA91573
:100AA000AF0A2F080A3C0319AF012F081E274B304D
:100AB0004B274E244A2D2C0E2D04023C031D872D5E
:100AC0002E08B7000319742DA9140230A906B70B1C
:100AD000662DA918742D02302F020319802D0630BF
:100AE0002F020319802D872DAF080319802D0430A4
:100AF0002F020319802D08302F020319802D872D16
:100B00002A0E2B040310293C03189D2D2D2D2C0E8D
:100B10002D040310123C031C2D2D2C08013C03193D
:100B2000932D1D30942D27302D070C20B3002A0E55
:100B30002B0403103302031C2D2D3A270C304427BD
:100B40004830152747304B27B73035070C2015277D
:100B50004E24071CB02D871D802C871C802CA92DAE
:100B6000A915B50A3508073C0319B50147304B27CD
:100B7000B73035070C2015274E24A92D2A081E272B
:100B80002B081E272F303D272C081E272D081E2737
:100B90002F303D272E081E272F081E2708008B12F6
:100BA000291000304B2721081E2722081E273A3023
:100BB0003D2723081E2724081E272030A91AEB30C2
:100BC0003D2740304B2740083D273F081E27390866
:100BD0001E272C303D2738081E27DF303D274330A5
:100BE0003D2748304B27BE2507304B27B730350708
:100BF0000C2015278B160800622683161E08831208
:100C0000C1001E08003C03190E2E1E08013C0319EA
:100C1000202E1E08023C03192F2E382E2D30C00026
:100C20000230BF000530B9000630B8004108031992
:100C300008004126C10B192E6D268A157421080063
:100C40002B30C000B801B901BF01410803190800E9
:100C50005126C10B282E6D268A15742108002B30D1
:100C6000C0000230BF000530B9000630B800252EA4
:100C70002B30C0000530BF000130B9000230B80091
:100C8000252EB803FF303802031D08000930B800D4
:100C9000B903FF303902031D08000930B900BF0352
:100CA0000800B80A0A303802031D0800B801B90A62
:100CB0000A303902031D0800B901BF0A08000A16EC
:100CC0005C240800C1309F001530B000B00B662EC8
:100CD0001F151F19692E1F100800123076270310E8
:100CE00040020319762E0318C12E952E40082D3C84
:100CF0000319A62E0B30762703103F020319832E0B
:100D00000318952EC12E0C307627031039020319D3
:100D10008C2E0318952EC12E0D3076270310380225
:100D2000031908000318952EC12E4008C300123085
:100D30005A273F08C3000B305A273908C3000C302C
:100D40005A273808C3000D305A2708000B30762781
:100D500003103F020319AF2E031C952EC12E0C3039
:100D60007627031039020319B82E031C952EC12EC5
:100D70000D3076270310380203190800031C952E46
:100D8000C12E13307627031040020319CA2E031810
:100D9000E92E080040082D3C0319FA2E0F30762763
:100DA00003103F020319D72E03180800E92E103054
:100DB0007627031039020319E02E03180800E92EE4
:100DC00011307627031038020319080003180800B1
:100DD000E92E4008C30013305A273F08C3000F30E4
:100DE0005A273908C30010305A273808C300113079
:100DF0005A2708000F30762703103F020319032FEC
:100E0000031C0800E92E103076270310390203195D
:100E10000C2F031C0800E92E11307627031038022E
:100E200003190800031C0800E92EA0000C20003E56
:100E3000031908003D27A00A2008162F303E3D2741
:100E400008008316FF308600831287178712071762
:100E5000FF308600861B2A2F8713071386138316FD
:100E6000860183120800383044270C3044270630AE
:100E70004427080001304427080087178716071306
:100E8000860087132127080087178712071386001B
:100E9000871321270800803844270800B000FF305E
:100EA000B100FF30B200B20B532FB10B512FB00B7A
:100EB0004F2F08008B13031783128D000313430871
:100EC00003178C0083168C130C1555308D00AA3037
:100ED0008D008C14831203138B170D1E6D2F831638
:100EE00003170C11831203130D1208008B13031741
:100EF00083128D0083168C130C1483120C080313B9
:100F00008B1708003F08C3000B305A270F305A27B1
:100F10003908C3000C305A2710305A273808C3004C
:100F20000D305A2711305A27FF30C3000E305A2790
:100F30004008C30012305A2713305A2708002108EE
:100F4000C30000305A272208C30001305A27230863
:100F5000C30002305A272408C30003305A272A0846
:100F6000C30004305A272B08C30005305A272C0829
:100F7000C30006305A272D08C30007305A272E0811
:100F8000C30008305A272F08C30009305A273508F4
:100F9000C3000A305A27291108008A1500288A152B
:100FA0002B2F0A168E280A16E3280A1638290A1645
:100FB0008D290A16E2290A16372A0A168C2AFF3FBB
:100FC000FF3FFF3FFF3FFF3FFF3FFF3FFF3FFF3F31
:100FD000FF3FFF3FFF3FFF3FFF3FFF3FFF3FFF3F21
:100FE000FF3FFF3FFF3FFF3FFF3FFF3FFF3FFF3F11
:100FF000FF3FFF3FFF3FFF3FFF3FFF3FFF3FFF3F01
:10100000A9113508C500C50803191628C503031919
:101010004828C50303197A28C5030319AC28C5035A
:101020000319DE28C5030319102942294008C3000B
:10103000163003271A3003273F08C3001730032751
:101040001B3003273908C300183003271C3003273F
:101050003808C300193003271D3003272108C300B7
:101060004E300327523003272208C3004F30032796
:10107000533003272308C30050300327543003277D
:101080002408C30051300327553003278A11080074
:101090004008C3001E300327223003273F08C30047
:1010A0001F300327233003273908C30020300327CC
:1010B000243003273808C3002130032725300327B5
:1010C0002108C300563003275A3003272208C300E3
:1010D000573003275B3003272308C300583003270A
:1010E0005C3003272408C300593003275D300327F1
:1010F0008A1108004008C300263003272A3003273E
:101100003F08C300273003272B3003273908C300CB
:10111000283003272C3003273808C3002930032741
:101120002D3003272108C3005E30032762300327D8
:101130002208C3005F300327633003272308C3005E
:1011400060300327643003272408C300613003277D
:10115000653003278A1108004008C3002E3003279A
:10116000323003273F08C3002F30032733300327D3
:101170003908C30030300327343003273808C30050
:1011800031300327353003272108C3006630032799
:101190006A3003272208C300673003276B30032718
:1011A0002308C300683003276C3003272408C300DA
:1011B000693003276D3003278A1108004008C300F7
:1011C000363003273A3003273F08C3003730032760
:1011D0003B3003273908C300383003273C3003274E
:1011E0003808C300393003273D3003272108C300E6
:1011F0006E300327723003272208C3006F300327A5
:10120000733003272308C30070300327743003278B
:101210002408C30071300327753003278A110800A2
:101220004008C3003E300327423003273F08C30075
:101230003F300327433003273908C30040300327DA
:10124000443003273808C3004130032745300327C3
:101250002108C300763003277A3003272208C30011
:10126000773003277B3003272308C3007830032718
:101270007C3003272408C300793003277D300327FF
:101280008A1108004008C300463003274A3003276C
:101290003F08C300473003274B3003273908C300FA
:1012A000483003274C3003273808C3004930032750
:1012B0004D3003272108C3007E30032782300327E7
:1012C0002208C3007F300327833003272308C3008D
:1012D00080300327843003272408C300813003278C
:1012E000853003278A1108003508C500C508031991
:1012F0008929C5030319532AC50303191B2BC503E9
:101300000319E32BC5030319AB2CC5030319732D74
:101310003B2E16301F270310400203199229031891
:10132000ED29B12940082D3C0319D22917301F2778
:1013300003103F0203199F290318B129ED29183022
:101340001F27031039020319A8290318B129ED2911
:1013500019301F27031038020319512A0318B12925
:10136000ED294008C300163003273F08C30017309B
:1013700003273908C300183003273808C300193081
:1013800003272108C3004E3003272208C3004F3033
:1013900003272308C300503003272408C30051301B
:1013A0000327512A17301F2703103F020319DB2997
:1013B000031CB129ED2918301F2703103902031926
:1013C000E429031CB129ED2919301F270310380225
:1013D0000319512A031CB129ED291A301F270310C4
:1013E00040020319F6290318152A512A40082D3CFA
:1013F0000319362A1B301F2703103F020319032A43
:101400000318512A152A1C301F270310390203190B
:101410000C2A0318512A152A1D301F2703103802E1
:101420000319512A0318512A152A4008C3001A30FB
:1014300003273F08C3001B3003273908C3001C30B3
:1014400003273808C3001D3003272108C30052308A
:1014500003272208C300533003272308C300543056
:1014600003272408C30055300327512A1B301F27A8
:1014700003103F0203193F2A031C512A152A1C306E
:101480001F27031039020319482A031C512A152A61
:101490001D301F27031038020319512A031C512A3B
:1014A000152A8A1108001E301F2703104002031955
:1014B0005C2A0318B72A7B2A40082D3C03199C2A72
:1014C0001F301F2703103F020319692A03187B2AC4
:1014D000B72A20301F27031039020319722A031874
:1014E0007B2AB72A21301F27031038020319512AFB
:1014F00003187B2AB72A4008C3001E3003273F0881
:10150000C3001F3003273908C300203003273808E1
:10151000C300213003272108C300563003272208C7
:10152000C300573003272308C3005830032724087B
:10153000C30059300327512A1F301F2703103F02D1
:101540000319A52A031C7B2AB72A20301F27031062
:1015500039020319E429031C7B2AB72A21301F27EB
:10156000031038020319512A031C7B2AB72A2230A0
:101570001F27031040020319C02A0318DF2A512A2B
:1015800040082D3C0319002B23301F2703103F0276
:101590000319CD2A0318512ADF2A24301F270310EC
:1015A00039020319D62A0318512ADF2A25301F27AA
:1015B000031038020319512A0318512ADF2A400860
:1015C000C300223003273F08C30023300327390814
:1015D000C300243003273808C3002530032721081F
:1015E000C3005A3003272208C3005B3003272308B7
:1015F000C3005C3003272408C3005D300327512A51
:1016000023301F2703103F020319092B031C512A03
:10161000DF2A24301F27031039020319122B031C61
:10162000512ADF2A25301F27031038020319512AB7
:10163000031C512ADF2A26301F27031040020319FA
:10164000242B03187F2B432B40082D3C0319642BBC
:1016500027301F2703103F020319312B0318432B98
:101660007F2B28301F270310390203193A2B031848
:10167000432B7F2B29301F27031038020319512ACF
:101680000318432B7F2B4008C300263003273F0855
:10169000C300273003273908C30028300327380840
:1016A000C300293003272108C3005E300327220826
:1016B000C3005F3003272308C300603003272408DA
:1016C000C30061300327512A27301F2703103F0230
:1016D00003196D2B031C432B7F2B28301F2703106E
:1016E00039020319762B031C432B7F2B29301F272C
:1016F000031038020319512A031C432B7F2B2A3075
:101700001F27031040020319882B0318A72B512A07
:1017100040082D3C0319C82B2B301F2703103F0214
:101720000319952B0318512AA72B2C301F270310C0
:10173000390203199E2B0318512AA72B2D301F277E
:10174000031038020319512A0318512AA72B400805
:10175000C3002A3003273F08C3002B300327390872
:10176000C3002C3003273808C3002D30032721087D
:10177000C300623003272208C30063300327230815
:10178000C300643003272408C30065300327512AAF
:101790002B301F2703103F020319D12B031C512AA2
:1017A000A72B2C301F27031039020319DA2B031C37
:1017B000512AA72B2D301F27031038020319512A55
:1017C000031C512AA72B2E301F2703104002031998
:1017D000EC2B0318472C0B2C40082D3C03192C2C08
:1017E0002F301F2703103F020319F92B03180B2C6E
:1017F000472C30301F27031039020319022C03181D
:101800000B2C472C31301F27031038020319512AA3
:1018100003180B2C472C4008C3002E3003273F0829
:10182000C3002F3003273908C3003030032738089E
:10183000C300313003272108C30066300327220884
:10184000C300673003272308C30068300327240838
:10185000C30069300327512A2F301F2703103F028E
:101860000319352C031C0B2C472C30301F27031079
:10187000390203193E2C031C0B2C472C31301F2737
:10188000031038020319512A031C0B2C472C323049
:101890001F27031040020319502C03186F2C512AE4
:1018A00040082D3C0319902C33301F2703103F02B2
:1018B00003195D2C0318512A6F2C34301F27031095
:1018C00039020319662C0318512A6F2C35301F2753
:1018D000031038020319512A0318512A6F2C4008AB
:1018E000C300323003273F08C300333003273908D1
:1018F000C300343003273808C300353003272108DC
:10190000C3006A3003272208C3006B300327230873
:10191000C3006C3003272408C3006D300327512A0D
:1019200033301F2703103F020319992C031C512A3F
:101930006F2C34301F27031039020319A22C031C0B
:10194000512A6F2C35301F27031038020319512AF2
:10195000031C512A6F2C36301F2703104002031935
:10196000B42C03180F2DD32C40082D3C0319F42C54
:1019700037301F2703103F020319C12C0318D32C43
:101980000F2D38301F27031039020319CA2C0318F2
:10199000D32C0F2D39301F27031038020319512A79
:1019A0000318D32C0F2D4008C300363003273F08FF
:1019B000C300373003273908C300383003273808FD
:1019C000C300393003272108C3006E3003272208E3
:1019D000C3006F3003272308C30070300327240897
:1019E000C30071300327512A37301F2703103F02ED
:1019F0000319FD2C031CD32C0F2D38301F27031087
:101A000039020319062D031CD32C0F2D39301F2743
:101A1000031038020319512A031CD32C0F2D3A301E
:101A20001F27031040020319182D0318372D512AC0
:101A300040082D3C0319582D3B301F2703103F024F
:101A40000319252D0318512A372D3C301F27031069
:101A5000390203192E2D0318512A372D3D301F2727
:101A6000031038020319512A0318512A372D400850
:101A7000C3003A3003273F08C3003B30032739082F
:101A8000C3003C3003273808C3003D30032721083A
:101A9000C300723003272208C300733003272308D2
:101AA000C300743003272408C30075300327512A6C
:101AB0003B301F2703103F020319612D031C512ADD
:101AC000372D3C301F270310390203196A2D031CE0
:101AD000512A372D3D301F27031038020319512A90
:101AE000031C512A372D3E301F27031040020319D3
:101AF0007C2D0318D72D9B2D40082D3C0319BC2DA0
:101B00003F301F2703103F020319892D03189B2D17
:101B1000D72D40301F27031039020319922D0318C7
:101B20009B2DD72D41301F27031038020319512A4E
:101B300003189B2DD72D4008C3003E3003273F08D4
:101B4000C3003F3003273908C3004030032738085B
:101B5000C300413003272108C30076300327220841
:101B6000C300773003272308C300783003272408F5
:101B7000C30079300327512A3F301F2703103F024B
:101B80000319C52D031C9B2DD72D40301F27031093
:101B900039020319CE2D031C9B2DD72D41301F2751
:101BA000031038020319512A031C9B2DD72D4230F4
:101BB0001F27031040020319E02D0318FF2D512A9F
:101BC00040082D3C0319202E43301F2703103F02ED
:101BD0000319ED2D0318512AFF2D44301F27031040
:101BE00039020319F62D0318512AFF2D45301F27FE
:101BF000031038020319512A0318512AFF2D4008F7
:101C0000C300423003273F08C3004330032739088D
:101C1000C300443003273808C30045300327210898
:101C2000C3007A3003272208C3007B300327230830
:101C3000C3007C3003272408C3007D300327512ACA
:101C400043301F2703103F020319292E031C512A7A
:101C5000FF2D44301F27031039020319322E031CB5
:101C6000512AFF2D45301F27031038020319512A2E
:101C7000031C512AFF2D46301F2703104002031971
:101C8000442E03189F2E632E40082D3C0319842EEA
:101C900047301F2703103F020319512E0318632EEC
:101CA0009F2E48301F270310390203195A2E03189C
:101CB000632E9F2E49301F27031038020319512A23
:101CC0000318632E9F2E4008C300463003273F08A9
:101CD000C300473003273908C300483003273808BA
:101CE000C300493003272108C3007E3003272208A0
:101CF000C3007F3003272308C30080300327240854
:101D0000C30081300327512A47301F2703103F02A9
:101D100003198D2E031C632E9F2E48301F2703109E
:101D200039020319962E031C632E9F2E49301F275C
:101D3000031038020319512A031C632E9F2E4A30C8
:101D40001F27031040020319A82E0318C72E512A7B
:101D500040082D3C0319E82E4B301F2703103F028B
:101D60000319B52E0318512AC72E4C301F27031014
:101D700039020319BE2E0318512AC72E4D301F27D2
:101D8000031038020319512A0318512AC72E40089C
:101D9000C3004A3003273F08C3004B3003273908EC
:101DA000C3004C3003273808C3004D3003272108F7
:101DB000C300823003272208C3008330032723088F
:101DC000C300843003272408C30085300327512A29
:101DD0004B301F2703103F020319F12E031C512A19
:101DE000C72E4C301F27031039020319FA2E031C8B
:101DF000512AC72E4D301F27031038020319512ACC
:101E0000031C512AC72E8B13031783128D00031353
:101E1000430803178C0083168C130C1555308D0066
:101E2000AA308D008C14831203138B170D1E162FEE
:101E3000831603170C11831203130D1208008B1362
:101E4000031783128D0083168C130C1483120C0855
:101E500003138B17080095274D309827413098279A
:101E6000583098272030982716301F27982717308A
:101E70001F27A92718301F27A9272C30982719308A
:101E80001F27A9270B30A6274E301F27A9274F3021
:101E90001F27A9273A30982750301F27A9275130EC
:101EA0001F27A9274030A6274D309827493098276B
:101EB0004E309827203098271A301F2798271B303C
:101EC0001F27A9271C301F27A9272C3098271D3032
:101ED0001F27A9274B30A62752301F27A927533089
:101EE0001F27A9273A30982754301F27A927553094
:101EF0001F27A92780275214871D7B2F8A11942919
:101F0000521407080B39B100EF30D100D10B892FE3
:101F10000800EF30B000B00B8B2F07080B393102EF
:101F2000B000B00AB00B802F862F01309F27080029
:101F300087178716071386008713AC2708008717B3
:101F40008712071386008713AC27080080389F2765
:101F50000800303E982708008316FF308600831261
:101F6000871787120717FF308600861BB52F871348
:101F7000071386138316860183120800FF3FFF3F75
:101F8000FF3FFF3FFF3FFF3FFF3FFF3FFF3FFF3F61
:101F9000FF3FFF3FFF3FFF3FFF3FFF3FFF3FFF3F51
:101FA000FF3FFF3FFF3FFF3FFF3FFF3FFF3FFF3F41
:101FB000FF3FFF3FFF3FFF3FFF3FFF3FFF3FFF3F31
:101FC000FF3FFF3FFF3FFF3FFF3FFF3FFF3FFF3F21
:101FD000FF3FFF3FFF3FFF3FFF3FFF3FFF3FFF3F11
:101FE000FF3FFF3FFF3FFF3FFF3FFF3FFF3FFF3F01
:101FF000FF3FFF3FFF3FFF3FFF3FFF3FFF3FFF3FF1
:1020000082005434653472346D346F346D34653409
:10201000743472346F342034763432342E343034A5
:10202000003450346F3472342034433461347234A9
:102030006C346F34733420344434693461347A340A
:10204000003468347434743470343A342F342F3498
:102050007734773477342E3465346C3465346334B4
:102060007434003472346F346E342E346534733407
:102070002E34763467342034203420342034203415
:1020800020342034003441346C34613472346D3483
:1020900061342034003449346C3475346D3469341F
:1020A0006E3461347234203444346934733470349F
:1020B0006C346134793400344134553454344F3401
:1020C0002034313400344134553454344F342034C6
:1020D000323400345334493445344D34503452345E
:1020E000453400344E3455344E3443344134203476
:1020F00020340034AE230130EC234030BF231130B4
:10210000EC232530F523AE232130EC234030BF23D0
:102110003230EC235030F5230A120800AE234D3044
:10212000B1234130B1235830B1232030B1231E30C8
:10213000A223B1231F30A223C2232030A223C22313
:102140002C30B1232130A223C2230B30BF235630C1
:10215000A223C2235730A223C2233A30B1235830DE
:10216000A223C2235930A223C2234030BF234D30C3
:10217000B1234930B1234E30B1232030B123223076
:10218000A223B1232330A223C2232430A223C223BB
:102190002C30B1232530A223C2234B30BF235A3029
:1021A000A223C2235B30A223C2233A30B1235C3086
:1021B000A223C2235D30A223C223D7235214871D3A
:1021C000DE280A12D329AE234D30B1234130B1238A
:1021D0005830B1232030B1232630A223B123273039
:1021E000A223C2232830A223C2232C30B1232930BA
:1021F000A223C2230B30BF235E30A223C2235F3051
:10220000A223C2233A30B1236030A223C22361301B
:10221000A223C2234030BF234D30B1234930B12324
:102220004E30B1232030B1232A30A223B1232B30EA
:10223000A223C2232C30A223C2232C30B1232D3061
:10224000A223C2234B30BF236230A223C2236330B8
:10225000A223C2233A30B1236430A223C2236530C3
:10226000A223C223D7235214871D33290A12122A0C
:10227000AE234D30B1234130B1235830B12320304B
:10228000B1232E30A223B1232F30A223C22330301A
:10229000A223C2232C30B1233130A223C2230B301E
:1022A000BF236630A223C2236730A223C2233A3061
:1022B000B1236830A223C2236930A223C223403055
:1022C000BF234D30B1234930B1234E30B1232030EC
:1022D000B1233230A223B1233330A223C2233430BE
:1022E000A223C2232C30B1233530A223C2234B308A
:1022F000BF236A30A223C2236B30A223C2233A3009
:10230000B1236C30A223C2236D30A223C223D72372
:102310005214871D88290A12512AAE234D30B12349
:102320004130B1235830B1232030B1233630A223BD
:10233000B1233730A223C2233830A223C2232C304A
:10234000B1233930A223C2230B30BF236E30A22326
:10235000C2236F30A223C2233A30B1237030A223AC
:10236000C2237130A223C2234030BF234D30B1239A
:102370004930B1234E30B1232030B1233A30A2236B
:10238000B1233B30A223C2233C30A223C2232C30F2
:10239000B1233D30A223C2234B30BF237230A2238E
:1023A000C2237330A223C2233A30B1237430A22354
:1023B000C2237530A223C223D7235214871DDD29DF
:1023C0000A12902AAE234D30B1234130B123583048
:1023D000B1232030B1233E30A223B1233F30A223CA
:1023E000C2234030A223C2232C30B1234130A22388
:1023F000C2230B30BF237630A223C2237730A2231F
:10240000C2233A30B1237830A223C2237930A223E9
:10241000C2234030BF234D30B1234930B1234E3069
:10242000B1232030B1234230A223B1234330A22371
:10243000C2234430A223C2232C30B1234530A2232F
:10244000C2234B30BF237A30A223C2237B30A22386
:10245000C2233A30B1237C30A223C2237D30A22391
:10246000C223D7235214871D322A0A12CF2AAE2341
:102470004D30B1234130B1235830B1232030B12346
:102480004630A223B1234730A223C2234830A223DF
:10249000C2232C30B1234930A223C2230B30BF23E7
:1024A0007E30A223C2237F30A223C2233A30B1233D
:1024B0008030A223C2238130A223C2234030BF2315
:1024C0004D30B1234930B1234E30B1232030B123F8
:1024D0004A30A223B1234B30A223C2234C30A22383
:1024E000C2232C30B1234D30A223C2234B30BF2353
:1024F0008230A223C2238330A223C2233A30B123E5
:102500008430A223C2238530A223C223D7235214AE
:10251000871D872A0A120E2BAE230230BF234330B9
:10252000EC23A91E952A9023962A85234530BF23A4
:102530008630A223C2238730A223C2233A30B1239C
:102540008830A223C2238930A223C2230124EF3082
:10255000C400FF30B100FF303230071CBA2A871D9B
:10256000C62A871C9B2BB20BAD2AB10BAB2AC40B1E
:10257000A92A9F2B29172030A9060930BF23FF3035
:10258000C300A91EC3018A300A24912A2917D72320
:102590000730B000FF30B100FF30B2008719A72A22
:1025A000B20BCE2AB10BCC2AB00BCA2A4530BF23BE
:1025B0000E30B8230124A912071C2D23871CE32AFF
:1025C000871D012BDB2A4630BF230124071C3F2334
:1025D000871CED2A871D012BE62A4830BF230124E2
:1025E000071C5123871CF72A871D012BF02A49302D
:1025F000BF230124071C6323871C012B871D012B8C
:10260000FA2A0C30B8238630A223C900C90E8730BD
:10261000A223C9042430031049020318162B1B23DC
:10262000A916FF30C3008A300A248C2A7923752327
:102630001B23A9128C2A2023080020230A12080039
:102640008630A223BA008730A223BB008830A223A1
:10265000BC008930A223BD0008008630A223013EC1
:10266000C30086300A248630A223033C0319752355
:102670008630A223C2234530BF23012408008730BF
:10268000A223013EC30087300A248730A2230A3CDC
:10269000031979238730A223C2234630BF230124A4
:1026A00008008830A223013EC30088300A24883005
:1026B000A223063C03197D238830A223C22348307D
:1026C000BF23012408008930A223013EC3008930C2
:1026D0000A248930A2230A3C031981238930A223CA
:1026E000C2234930BF2301240800C30186300A24D5
:1026F0000800C30187300A240800C30188300A2477
:102700000800C30189300A2408002830B1234F3063
:10271000B1234630B1234630B1232930B12308001C
:102720002830B1234F30B1234E30B1232930B123AB
:102730002030B1230800291B9F2B0A12602B29137C
:102740000A1231298B13031783128D0083168C1301
:102750000C1483120C0803138B1708000130B823E4
:10276000080087178716071386008713C5230800FC
:1027700087178712071386008713C5230800803840
:10278000B8230800303EB12308008316FF308600CE
:102790008312871787120717FF308600861BCE2B00
:1027A00087130713861383168601831208005214B9
:1027B00007080B39B100EF30D100D10BE02B080036
:1027C000EF30B000B00BE22B07080B393102B0003C
:1027D000B00AB00BD72BDD2BA0000020003E031960
:1027E0000800B123A00A2008ED2BB000FF30B10093
:1027F000FF30B200B20BFA2BB10BF82BB00BF62B5B
:102800000800D723871C022C871D042C071C062CCC
:10281000D72308008B13031783128D00031343087B
:1028200003178C0083168C130C1555308D00AA30BD
:102830008D008C14831203138B170D1E1D2C831611
:1028400003170C11831203130D1208003A0821021A
:10285000031D382C3B082202031D382C3C082302A0
:10286000031D382C3D082402031D382CA917382CD1
:102870000A12402CCC18442C0712CD0B8C28FF30A8
:10288000CD000230CC068C28CD0B4B2CFF30CD0078
:102890000230CC068C284C1C552C10308706CB0BF4
:1028A0008C280A30CB004C108C280712CA0B8C28BD
:1028B0000A30CA004C148C28521407080B39B10096
:1028C000EF30D100D10B662C0A120800EF30B000B7
:1028D000B00B682C07080B393102B000B00AB00BFE
:1028E0005C2C622C5219872CD219822C521A7A2C09
:1028F000D21A7E2CEF30D700D6008B2C0030D700B8
:10290000D6008B2C0030D700EF30D6008B2C503007
:10291000D700EF30D6005218A124D218A824902C4A
:1029200015080310530203189F2C9503D40B9D2CFC
:10293000D50B9D2C0F30D500D2140A128F2B950A7F
:102940009D2C52105608D300D4010F30D50008003A
:10295000D2105708D30008005214AE234B30EC239A
:102960005219B82CD219D02C521AE82CD21A002D98
:102970004030BF235C30EC230124EF30C400FF3033
:10298000B100FF303230871C182D071CD02C871D5A
:102990005214B20BC32CB10BC12CC40BBF2C242D71
:1029A0004030BF236330EC230124EF30C400FF30FC
:1029B000B100FF303230871C1A2D071CE82C871D10
:1029C0005214B20BDB2CB10BD92CC40BD72C242DF9
:1029D0004030BF236A30EC230124EF30C400FF30C5
:1029E000B100FF303230871C1C2D071C002D871DC5
:1029F0005214B20BF32CB10BF12CC40BEF2C242D81
:102A00004030BF237230EC230124EF30C400FF308C
:102A1000B100FF303230871C1E2D071CB82C871DDB
:102A20005214B20B0B2DB10B092DC40B072D242D05
:102A30000430202D0830202D1030202D2030202D66
:102A4000D200C3008B300A240A123129FF3FFF3F16
:102A5000FF3FFF3FFF3FFF3FFF3FFF3FFF3FFF3F86
:102A6000FF3FFF3FFF3FFF3FFF3FFF3FFF3FFF3F76
:102A7000FF3FFF3FFF3FFF3FFF3FFF3FFF3FFF3F66
:102A8000FF3FFF3FFF3FFF3FFF3FFF3FFF3FFF3F56
:02400E003A3F37
:1042000000000000000000000000010000000100AC
:10421000000000000000000000000000000000009E
:1042200000000000FF00FF00FF00FF002B00000067
:10423000000000002B000000000000002B00000028
:10424000000000002B000000000000002B00000018
:10425000000000002B000000000000002B00000008
:10426000000000002B000000000000002B000000F8
:10427000000000002B000000000000002B000000E8
:10428000000000002B000000000000002B000000D8
:10429000000000002B00000000000000FF00FF00F5
:1042A000FF00FF00FF00FF00FF00FF00FF00FF0016
:1042B000FF00FF00FF00FF00FF00FF00FF00FF0006
:1042C000FF00FF00FF00FF00FF00FF00FF00FF00F6
:1042D000FF00FF00FF00FF00FF00FF00FF00FF00E6
:1042E000FF00FF00FF00FF00FF00FF00FF00FF00D6
:1042F000FF00FF00FF00FF00FF00FF00FF00FF00C6
:10430000FF00FF00FF00FF00FF00FF0000000000B3
:104310000000000000000500FF00FF00FF00FF009C
:10432000FF00FF00FF00FF00FF00FF00FF00FF0095
:10433000FF00FF00FF00FF00FF00FF00FF00FF0085
:10434000FF00FF00FF00FF00FF00FF00FF00FF0075
:10435000FF00FF00FF00FF00FF00FF00FF00FF0065
:10436000FF00FF00FF00FF00FF00FF00FF00FF0055
:10437000FF00FF00FF00FF00FF00FF00FF00FF0045
:10438000FF00FF00FF00FF00FF00FF00FF00FF0035
:10439000FF00FF00FF00FF00FF00FF00FF00FF0025
:1043A000FF00FF00FF00FF00FF00FF00FF00FF0015
:1043B000FF00FF00FF00FF00FF00FF00FF00FF0005
:1043C000FF00FF00FF00FF00FF00FF00FF00FF00F5
:1043D000FF00FF00FF00FF00FF00FF00FF00FF00E5
:1043E000FF00FF00FF00FF00FF00FF00FF00FF00D5
:1043F000FF00FF00FF00FF00FF00FF00FF00FF00C5
:00000001FF
